:100000000C9400050C9447050C940B080C944705C0
:100010000C9447050C9447050C9447050C94470530
:100020000C9447050C9447050C9447050C94C40D9B
:100030000C94730E0C94B71C0C9447050C94470554
:100040000C9447050C9447050C9447050C942B1D04
:100050000C9447050C9447050C9447050C944705F0
:100060000C9447050C9447050C9447050C944705E0
:100070000C944705E00E020FF00F020FF00F470F30
:100080006A0FF00FBF0FD20FD012D012FF12FF1263
:100090005D139B13B515B515B413B515B514B5148B
:1000A0008915B515B515A015350C12132B141A802A
:1000B00024252668742E2A272122230815171C18A8
:1000C0001E1F202F3031692D39041607090A0B0D28
:1000D0000E0F33343228807C79781D1B06190511E8
:1000E00010363738757D647A2C7B7F8040413A53D7
:1000F0005455565F606157805C5D5E6642433C6765
:100100005A5B582962635980808080803B473D510B
:100110008080494A4B4C4D4E463E48804452453FB4
:10012000504F808080808080253032580A002530F2
:1001300032580A004572726F723A20253032580ADE
:1001400000456E640A0073253032583A7225303209
:10015000582000456E61626C6520627265616B3A81
:1001600020004B6579626F6172642049443A202512
:100170003032580A0049424D203437303420636F02
:100180006E7665727465720A00726275663A2066F0
:10019000756C6C0A00523A25303258253032580AB4
:1001A00000533A2530325820004B6579626F6172F6
:1001B000642073746172742E0A0055534220636F79
:1001C0006E666967757265642E0A000D0A696E694C
:1001D000740A003803490042004D00200034003703
:1001E000003000340020006B006500790062006F71
:1001F00000610072006400200063006F006E0076F2
:10020000006500720074006500720000000E037447
:10021000002E006D002E006B002E0000000403096C
:100220000409027400040100A03209040000010363
:10023000010100092111010001224000070581038D
:1002400008000A090401000103010200092111014B
:100250000001224D000705820308000A090402007C
:1002600001030000000921110100012236000705E9
:10027000830308000A0904030002030000000921A7
:100280001101000122220007058403200001070557
:1002900004032000011201100100000008EDFE0718
:1002A000470100010200010631FF0974A10109752F
:1002B000150026FF00952075088102097615002695
:1002C000FF00952075089102C005010980A10185F4
:1002D0000216810026B7001A81002AB70075109512
:1002E000018100C0050C0901A1018503160100264A
:1002F0009C021A01002A9C02751095018100C0051C
:10030000010902A1010901A1000509190129051529
:10031000002501950575018102950175038101058F
:1003200001093009311581257F950275088106097B
:10033000381581257F950175088106050C0A38025C
:100340001581257F950175088106C0C00501090644
:10035000A101050719E029E7150025019508750198
:100360008102950175088101050819012905950586
:10037000750191029501750391010507190029FF87
:10038000150026FF00950675088100C0636F6E7327
:10039000756D65723A20253034580A00737973748C
:1003A000656D3A20253034580A000A00253032584D
:1003B00020006B6579626F6172643A20004C45449D
:1003C0003A20253032580A00253032583A2025305C
:1003D000386225730A00722F63203031323334358E
:1003E00036370A00290A002575002F002575005DA3
:1003F00028002564002000256400200025640020DA
:10040000002564007C0025303258006D6F757365DF
:100410006B6579205B62746E7C7820792076206829
:100420005D287265702F61636C293A205B006D6BEB
:100430005F776865656C5F74696D655F746F5F6D2C
:100440006178203D2025640A006D6B5F77686565E3
:100450006C5F6D61785F7370656564203D20256415
:100460000A006D6B5F74696D655F746F5F6D6178B5
:10047000203D2025640A006D6B5F6D61785F7370AD
:10048000656564203D2025640A006D6B5F696E74AC
:10049000657276616C203D2025640A006D6B5F6497
:1004A000656C6179203D2025640A006D6B5F77687B
:1004B00065656C5F74696D655F746F5F6D617820F1
:1004C0003D2025640A006D6B5F776865656C5F6D24
:1004D00061785F7370656564203D2025640A006D56
:1004E0006B5F74696D655F746F5F6D6178203D202F
:1004F00025640A006D6B5F6D61785F73706565647C
:10050000203D2025640A006D6B5F696E746572760C
:10051000616C203D2025640A006D6B5F64656C6131
:1005200079203D2025640A000A00257500363A200E
:10053000776865656C5F74696D655F746F5F6D6129
:10054000783A20000A00257500353A2077686565FD
:100550006C5F6D61785F73706565643A20000A00B6
:10056000257500343A2074696D655F746F5F6D6145
:10057000783A20000A00257500333A206D61785FD3
:1005800073706565643A20000A00257500323A20D0
:10059000696E74657276616C286D73293A20000A61
:1005A00000257500313A2064656C6179282A313064
:1005B0006D73293A20000A092D2056616C75657308
:1005C000202D0A004D3E004D25643E20003F007363
:1005D00065742064656661756C740A00433E200092
:1005E00077686572652064656C74613A2063757222
:1005F000736F723D25642C20776865656C3D2564BA
:100600000A53656520687474703A2F2F656E2E77D3
:10061000696B6970656469612E6F72672F77696BAA
:10062000692F4D6F7573655F6B6579730A000A09F1
:100630002D204D6F7573656B6579202D0A455343E9
:100640002F713A09717569740A313A0964656C61F0
:1006500079282A31306D73290A323A09696E746536
:100660007276616C286D73290A333A096D61785F7F
:1006700073706565640A343A0974696D655F746FF7
:100680005F6D61780A353A09776865656C5F6D6101
:10069000785F73706565640A363A09776865656CDA
:1006A0005F74696D655F746F5F6D61780A0A703A97
:1006B000097072696E742076616C7565730A643AAC
:1006C000097365742064656661756C74730A75706E
:1006D0003A092B310A646F776E3A092D310A706737
:1006E00075703A092B31300A7067646F776E3A097A
:1006F0002D31300A0A7370656564203D2064656C95
:100700007461202A206D61785F7370656564202AAA
:100710002028726570656174202F2074696D655F93
:10072000746F5F6D6178290A003F004D3E200043E1
:100730003E20004C25640A000A092D20436F6E7389
:100740006F6C65202D0A4553432F713A0971756905
:10075000740A6D3A096D6F7573656B65790A000AE5
:10076000092D204D61676963202D0A643A0964658B
:100770006275670A783A096465627567206D61740D
:100780007269780A6B3A096465627567206B6579EE
:10079000626F6172640A6D3A096465627567206D03
:1007A0006F7573650A763A0976657273696F6E0ABA
:1007B000733A097374617475730A633A09636F6EEF
:1007C000736F6C65206D6F64650A302D343A096C67
:1007D00061796572302D34284631302D4634290A2E
:1007E000506175733A09626F6F746C6F6164657202
:1007F0000A003F0074696D65725F7265616433322F
:1008000028293A202530346C580A006B6579626FCC
:100810006172645F69646C653A2025580A006B65F3
:1008200079626F6172645F70726F746F636F6C3A3C
:100830002025580A00686F73745F6B6579626F6179
:1008400072645F6C65647328293A2025580A000A8F
:10085000092D20537461747573202D0A004743439A
:100860003A20342E392E32204156522D4C494243E3
:100870003A20312E382E3073766E204156525F4129
:100880005243483A2061767233350A004F5054493A
:100890004F4E533A204C554641204D4F5553454BF2
:1008A00045592045585452414B455920434F4E53CA
:1008B0004F4C4520434F4D4D414E44204B45594DE3
:1008C00041505F53454354494F4E20343039360A26
:1008D000004255494C443A20383238346433302D84
:1008E0006469727479202831363A33363A353220C9
:1008F0004170722032372032303138290A0056498F
:10090000443A2030784645454428742E6D2E6B2E8F
:1009100029205049443A203078343730372849422A
:100920004D2034373034206B6579626F61726420FA
:10093000636F6E76657274657229205645523A204F
:100940003078303030310A00444553433A20636FE9
:100950006E766572742049424D2034373034206BF6
:100960006579626F61726420746F205553420A008A
:100970000A092D2056657273696F6E202D0A000AD0
:100980006D6F7573653A206F66660A000A6D6F7544
:1009900073653A206F6E0A000A6B6579626F617247
:1009A000643A206F66660A000A6B6579626F61724D
:1009B000643A206F6E0A000A6D61747269783A2099
:1009C0006F66660A000A6D61747269783A206F6E0C
:1009D0000A000A64656275673A206F6E0A000A644D
:1009E000656275673A206F66660A000A0A626F6F71
:1009F000746C6F616465722E2E2E2000433E2000C1
:100A000011241FBECFEFD4E0DEBFCDBF04B603FE7E
:100A100027C08091780290917902A0917A02B091DA
:100A20007B028730904BA740B04BD1F410927802F4
:100A30001092790210927A0210927B0214BE84B74F
:100A4000877F84BF0FB6F894A89580916000886175
:100A500080936000109260000FBEE0E0F8E309951B
:100A600011E0A0E0B1E0E2E8FBE402C005900D92E5
:100A7000A233B107D9F722E0A2E3B1E001C01D9291
:100A8000A837B207E1F70E94050B0C94BF250C9420
:100A90000000FF93EF93E0913201F0913301309722
:100AA00009F00995EF91FF910895FC01859180303F
:100AB00011F0EFDFFBCF0895FF27E0E230E247FFC0
:100AC0000CC0419597FF09C0EDE260957095809547
:100AD0009095611D711D811D911D27FF02C02195FB
:100AE00030E350E2AA27660F771F881F991FAA1FBD
:100AF000A41710F0A41B63955A95A9F7AA3008F023
:100B0000A95FA05DAF93F39561157105810591050E
:100B100041F7ED3211F4EF93F395F21718F43F9388
:100B2000F395FBCF8F91B5DFFA95E1F70895E99141
:100B3000F9918591803021F0853219F0AADFF9CF43
:100B4000089520E0E89455915532C1F3503311F4E3
:100B5000689455915A3348F4505390F3220F022E63
:100B6000220F220F200D250FF4CF0EF4219589912D
:100B70009991533619F3533729F1533559F1BC0183
:100B800088279927E8945C3621F489919991689493
:100B90005591543639F446EF7EF077FF0DC08FEF54
:100BA0009FEF0AC055374AE039F0583540E121F04F
:100BB000523642E009F00895FF93EF937DDFEF9105
:100BC000FF91B7CFFF93EF93FC0181918030B9F390
:100BD00060DFFBCFFF93EF9368DFF1CFDF93CF931D
:100BE000CDB7DEB72596A3DFCF91DF9108950C94A2
:100BF0002A07E82FF0E0EC5CFE4F80810895E4E3E3
:100C0000F1E080E18E0F11928E13FDCF0895FF92D7
:100C10000F931F93CF93DF9380915A02816080934B
:100C20005A0285E791E00E9455050E94FF052FEFCB
:100C300087EA91E6215080409040E1F700C0000033
:100C40000E94FF071F928F9382E691E09F938F93FC
:100C50000E94EE0583E591E00E9455050F900F90EC
:100C60000F900F908CEF0E943907882339F08FE3A3
:100C70009CE90197F1F700C00000F4CFC0E0D0E09C
:100C800006E411E08C2F8068F82E8F2D0E94390722
:100C9000882339F08FE39CE90197F1F700C0000049
:100CA000F4CF8FE19EE40197F1F700C000000E94AD
:100CB000FF071F928F93DF93CF931F930F930E9491
:100CC000EE0521960F900F900F900F900F900F90C0
:100CD000CF37D105B9F68FEF0E943907882339F055
:100CE0008FE39CE90197F1F700C00000F4CF81E4A5
:100CF00091E0DF91CF911F910F91FF900C945505DA
:100D0000CF93DF930E94FF078F3F09F457C0982FBE
:100D10009F779C3778F01F928F9384E391E09F93A5
:100D20008F930E94EE050E94FF050F900F900F9089
:100D30000F9044C090915A02C82FC695C695C6958B
:100D4000D82FD77087FF1CC090FF0CC01F928F93C5
:100D50008EE291E09F938F930E94EE050F900F908B
:100D60000F900F90EC2FEF70F0E0EC5CFE4F81E005
:100D700090E001C0880FDA95EAF79081892B1BC0BB
:100D800090FF0CC01F928F9388E291E09F938F9306
:100D90000E94EE050F900F900F900F90EC2FF0E057
:100DA000EC5CFE4F81E090E001C0880FDA95EAF735
:100DB000809590818923808381E001C080E0DF916C
:100DC000CF91089508959FB7F8942091480180919C
:100DD0004901821761F030E0F901E65BFE4F808146
:100DE0002F5F3F4F2F7133272093480101C080E0D0
:100DF0009FBF08955198599A08955898509A089508
:100E00005098589A08955198599A85E08A95F1F723
:100E1000000089B18695817008955098589A85E0B0
:100E20008A95F1F7000089B181700895CF93DF931F
:100E3000C4E6D0E00E940307811108C0209731F07A
:100E400085E08A95F1F700002197F4CFCE01DF917C
:100E5000CF9108950E94FA060E94FD06E9E6F0E0AF
:100E600080818C608083E19AE99A0E94FA060C9452
:100E70000007BF92CF92DF92EF92FF920F931F93E2
:100E8000CF93DF93C82E10924701E9980E94FA068B
:100E90000E9400075998519A0CE211E00E940D0738
:100EA00081110AC00115110549F085E08A95F1F715
:100EB000000001501109F2CF012B11F480E373C03F
:100EC00000E010E0D1E0D12CBB24B394C02F0E94ED
:100ED0001607892B11F4C05C24C0C601002E02C085
:100EE000959587950A94E2F780FF04C0DB250E9460
:100EF000000702C00E94FD0684E6E82EF12C0E9445
:100F00000307882359F0E114F10451F085E08A9534
:100F1000F1F7000081E0E81AF108F1CFEF2821F4A1
:100F2000C85BC09347014AC00F5F1F4F08301105CF
:100F300069F60E941607892B11F484E334C0DD237F
:100F400029F00E94000704E610E00CC00E94FD0694
:100F5000FACF0115110561F085E08A95F1F70000DF
:100F6000015011090E9403078111F3CF012B11F4E5
:100F700085E319C00E941607892BF9F20E94000729
:100F800004E610E00E940D07882351F001151105B9
:100F900049F085E08A95F1F7000001501109F2CF80
:100FA000012B21F486E38093470108C00E94FA06D2
:100FB0000E940007E19AE99A80E017C00E94FA06B1
:100FC0000E94000780914701813360F01F928F9348
:100FD00081EA91E09F938F930E94EE050F900F900E
:100FE0000F900F90E19AE99A8FEFDF91CF911F91C7
:100FF0000F91FF90EF90DF90CF90BF9008952FB7A3
:10100000F89490914901809148012FBF98130C9456
:10101000E3068FEF08951F920F920FB60F921124DF
:101020002F933F934F935F936F937F938F939F93F0
:10103000AF93BF93CF93DF93EF93FF93109247014A
:10104000809146018830F1F030F0893009F05CC0C1
:10105000C4E6D0E02EC0809145018695809345017D
:101060000E940D07882309F449C0809145018068DA
:101070008093450181E090914401911180E080933B
:1010800044013CC00E940D07882339F081E0909113
:101090004401911180E080934401809144018823B0
:1010A00099F12CC0209781F185E08A95F1F7000035
:1010B00021970E940D078111F5CFCD2B29F1409189
:1010C0004501CFB7F8948091490190E09C012F5FD2
:1010D0003F4F2F71332750914801521739F0FC01CF
:1010E000E65BFE4F40832093490104C089E891E00C
:1010F0000E945505CFBF109247012AC0809146013A
:101100008F5F809346012AC08091460180934701FA
:101110008EEF0E943907882339F08FE99FE001970D
:10112000F1F700C00000F4CF809145011F928F932A
:10113000809146011F928F9385E991E09F938F9351
:101140000E94EE050F900F900F900F900F900F9050
:10115000109246011092450110924401FF91EF91C7
:10116000DF91CF91BF91AF919F918F917F916F91BF
:101170005F914F913F912F910F900FBE0F901F9055
:1011800018958091760108959FB7F89410926D019B
:101190009FBF90916F02943009F057C09091E90081
:1011A0009F703091EC00232F217030FD20E8922BAE
:1011B00024E02093E9002091EB0020FF43C0209120
:1011C000EE0027FF3FC020916A01222321F02091E9
:1011D000E80025FF37C010926A0126E03091E80050
:1011E00035FD15C030916F02343061F53091EB0060
:1011F00035FD28C0215021F481E080936A0122C08E
:10120000EFE9FFE03197F1F700C00000E7CF8093EE
:10121000F1008091E80085FD0AC08091E80080FF20
:10122000FCCF8091E8008E778093E80006C08FB7EE
:10123000F89421E020936D018FBF9F709093E90097
:1012400080E008959F709093E9008FEF0895CF9309
:10125000DF9300D01F92CDB7DEB79C0180916F0263
:10126000843019F593E099833B832A839093E900B6
:101270008FEF9091E800815095FD06C095ED9A950D
:10128000F1F700008111F5CF8091E80085FF0DC0D6
:1012900040E050E063E070E0CE0101960E94D20B86
:1012A0008091E8008E778093E8000F900F900F9068
:1012B000DF91CF910895CF93DF9300D01F92CDB7E8
:1012C000DEB720916F02243021F522E029839B8331
:1012D0008A8383E08093E9008FEF9091E80081504A
:1012E00095FD06C095ED9A95F1F700008111F5CFB7
:1012F0008091E80085FF0DC040E050E063E070E0C1
:10130000CE0101960E94D20B8091E8008E778093E7
:10131000E8000F900F900F90DF91CF9108952091EA
:101320006F022430F1F422E02093E9002FEF309196
:10133000E800215035FD06C035ED3A95F1F7000083
:101340002111F5CF2091E80025FF0BC040E050E0CF
:1013500065E070E00E94D20B8091E8008E77809368
:10136000E8000895CF93DF9320916F02243039F580
:1013700021E02093E9002FEF3091E800215035FD66
:1013800006C035ED3A95F1F700002111F5CF209117
:10139000E80025FF14C0EC0140E050E068E070E098
:1013A0000E94D20B8091E8008E778093E80088E05D
:1013B000FE01AEE6B1E001900D928A95E1F7DF9172
:1013C000CF910895089520916B012F5F822F62E3E2
:1013D0000E948525992319F020936B01089510929E
:1013E0006B0180916D01882371F180916F028430CF
:1013F00041F58091E9008F702091EC00922F91705F
:1014000020FD90E8892B94E09093E9009091EB0007
:1014100090FF14C09091EE0097FF10C09091E800EB
:1014200095FF03C01092F100F9CF9091E80090FF72
:1014300005C09091E8009E779093E8008F708093AC
:10144000E90010926D01089542E061EC81E00E9494
:10145000DB0C42E061EC82E00E94DB0C42E061ECDC
:1014600083E00E94DB0C42E261EC84E00C94DB0C34
:1014700080917102833009F453C030F4813071F0EF
:10148000823009F48CC008958A3009F478C08B301A
:1014900009F45EC0893009F09AC020C080917002C2
:1014A000813A09F094C08091E800877F8093E8003A
:1014B0008091740290917502892B21F468E08EE688
:1014C00091E003C060E080E090E070E00E941D0CBD
:1014D0008091E8008B778093E800089580917002F6
:1014E000813209F074C08091740290917502892B49
:1014F00009F06DC08091E800877F8093E8008091BB
:10150000E80082FD05C080916F028111F8CF5FC0B5
:101510008091F100809376018091E8008B7753C031
:1015200080917002813A09F052C0809174029091CA
:101530007502892B09F04BC08091E800877F80936A
:10154000E8008091E80080FFFCCF80910A0136C05E
:10155000809170028132D9F5809174029091750268
:10156000892BA9F58091E800877F8093E8000E948D
:10157000100D8091720280930A010C94D71580910E
:101580007002813221F58091E800877F8093E80026
:101590000E94100D809173028093770108958091CD
:1015A0007002813AA1F48091E800877F8093E8007F
:1015B0008091E80080FFFCCF809177018093F1005B
:1015C0008091E8008E778093E8000C94100D0895C8
:1015D000089508958091760180936C0110927601B0
:1015E00080E00E94E2060E94FF050C94D7150C943F
:1015F000EA0A0E94761C80916D02882329F00E94DD
:101600009F1C81110C94BC0B089584B7877F84BF05
:101610000FB6F894A895809160008861809360006F
:10162000109260000FBE90E080E80FB6F8948093AF
:101630006100909361000FBE84EC98E00E944B1C07
:101640008BEC91E00E9455050E94E80A0E94C910A7
:101650000E94610D0E94B40D8091E200846080932D
:10166000E200789480916F028430E1F781ED97E099
:10167000019739F0EFE9FFE03197F1F700C0000082
:10168000F7CF8AEB91E00E9455050E94CB1080E0D5
:1016900091E00E94081089EA91E00E9455050E949D
:1016A000E90A80916F02853019F40E94F90AF9CF96
:1016B0000E94CF10F6CF0E94B31C80916C018093E2
:1016C000760108950C945B0B292F332723303105C5
:1016D000C9F064F42130310581F02230310509F080
:1016E00043C084E790E021E232E042C0213231057C
:1016F000F1F02232310541F137C082E190E025E975
:1017000032E036C099278130910541F08230910551
:1017100041F0892B49F5EDE1F2E005C0EDE0F2E0A2
:1017200002C0E3EDF1E0849190E09F0121C06430BC
:10173000D8F4E62FF0E0EE0FFF1FE15EFE4F2081B0
:10174000318189E090E014C0643070F470E0FB01F6
:10175000EE0FFF1FE95EFE4F20813181FB01ED5E40
:10176000FE4F808190E004C080E090E020E030E017
:10177000FA0131832083089584E089BD86E089BD24
:1017800009B400FEFDCF8091D8008F7D8093D800F2
:101790008091E00082608093E0008091E00081FD14
:1017A000FCCF0895CF92DF92EF92FF920F931F9399
:1017B000CF93DF93EC018B016A010E942F0D811101
:1017C00033C0C114D10439F0F60180819181081B26
:1017D000190BC80FD91FE12CF12C0115110519F1B6
:1017E0008091E80085FD16C08091E8008E77809397
:1017F000E800C114D10449F0F60180819181E80E1E
:10180000F91EF182E08285E00FC00E942F0D88232F
:1018100021F30AC089918093F10001501109FFEF73
:10182000EF1AFF0ADACF80E0DF91CF911F910F917D
:10183000FF90EF90DF90CF90089520917602309145
:1018400077022617370748F06115710539F42091A2
:10185000E8002E772093E80001C0B90140E061154F
:10186000710591F120916F02222309F440C02530C7
:1018700009F43FC02091E80023FD3DC02091E8001D
:1018800022FD2FC02091E80020FFE9CF2091F20037
:1018900030E0FC01CF016115710559F028303105A8
:1018A00040F481918093F100615071092F5F3F4FA7
:1018B000F1CF41E02830310509F040E02091E80007
:1018C0002E772093E800CBCF4111CCCF0AC0809176
:1018D0006F02882361F0853061F08091E80083FD1C
:1018E0000AC08091E80082FFF2CF80E0089582E094
:1018F000089583E0089581E0089520917602309163
:1019000077022617370748F06115710539F42091E1
:10191000E8002E772093E80001C0B901FC0120E027
:101920006115710579F180916F02882309F43DC03A
:10193000853009F43CC08091E80083FD3AC0809175
:10194000E80082FD2CC08091E80080FFE9CF809103
:10195000F20090E06115710559F08830910540F46E
:1019600024912093F1003196615071090196F2CFD4
:1019700021E0089709F020E08091E8008E778093BD
:10198000E800CECF2111CFCF0AC080916F0288230B
:1019900061F0853061F08091E80083FD0AC080919C
:1019A000E80082FFF2CF80E0089582E0089583E0AE
:1019B000089581E00895982F953058F59093E900A7
:1019C000981739F07091EC002091ED005091F000E3
:1019D00003C0242F762F50E021FF19C03091EB0077
:1019E0003E7F3093EB003091ED003D7F3093ED0072
:1019F0003091EB0031603093EB007093EC0020935A
:101A0000ED005093F0002091EE0027FF07C09F5F8C
:101A1000D3CF8F708093E90081E0089580E008952E
:101A20008091700287FF11C08091E80082FD05C09F
:101A300080916F028111F8CF11C08091E8008B77FF
:101A40000BC080916F02882349F08091E80080FFED
:101A5000F8CF8091E8008E778093E8000895209178
:101A6000E4003091E50095E64091EC00842F817010
:101A700040FF22C08091E80080FD1CC080916F0271
:101A8000882391F0853091F08091EB0085FD10C0A6
:101A90004091E4005091E5004217530729F39A0161
:101AA000915011F784E0089582E0089583E008954D
:101AB00081E0089580E008954091E80042FFDECF84
:101AC00008950E94BE0D0E94C10DE0EEF0E08081FD
:101AD00081608083E8EDF0E080818F77808319BC9E
:101AE000E3E6F0E080818160808310926E020895C9
:101AF0000E94BE0D0E94C10D8091D8008F77809307
:101B0000D8008091D80080688093D8008091D80058
:101B10008F7D8093D80084E089BD86E089BD09B4BB
:101B200000FEFDCF10926F0210926B0210926D02B8
:101B300010926C0242E060E080E00E94DB0C809139
:101B4000E1008E7F8093E1008091E20081608093CC
:101B5000E2008091E20088608093E2008091E000E2
:101B60008E7F8093E0000895E3E6F0E080818E7F31
:101B7000808381E080936E020C94780D1092E200D5
:101B800008951092E10008951F920F920FB60F92E0
:101B900011242F933F934F935F936F937F938F9372
:101BA0009F93AF93BF93EF93FF938091E10082FFE8
:101BB0000BC08091E20082FF07C08091E1008B7F23
:101BC0008093E1000E94E3098091E10080FF19C049
:101BD0008091E20080FF15C08091E2008E7F8093AB
:101BE000E2008091E20080618093E2008091D80061
:101BF00080628093D80019BC85E080936F020E94B8
:101C0000F70A8091E10084FF30C08091E20084FFF8
:101C10002CC084E089BD86E089BD09B400FEFDCFFB
:101C20008091D8008F7D8093D8008091E1008F7ED5
:101C30008093E1008091E2008F7E8093E2008091AA
:101C4000E20081608093E20080916B02882311F0B2
:101C500084E007C08091E30087FD02C081E001C0FD
:101C600083E080936F020E94620B8091E10083FF0A
:101C700029C08091E20083FF25C08091E100877F29
:101C80008093E10082E080936F0210926B0280915A
:101C9000E1008E7F8093E1008091E2008E7F80934F
:101CA000E2008091E20080618093E20042E060E027
:101CB00080E00E94DB0C8091F00088608093F0004F
:101CC0000E94E209FF91EF91BF91AF919F918F9197
:101CD0007F916F915F914F913F912F910F900FBE28
:101CE0000F901F9018951F920F920FB60F9211240C
:101CF0002F933F934F935F936F937F938F939F9314
:101D0000AF93BF93CF93DF93EF93FF93C091E9001D
:101D1000CF708091EC00D82FD17080FDD0E8109268
:101D2000E9008091F000877F8093F00078940E9412
:101D3000B70E1092E9008091F00088608093F00067
:101D4000CD2BCF70C093E900FF91EF91DF91CF9140
:101D5000BF91AF919F918F917F916F915F914F91C3
:101D60003F912F910F900FBE0F901F9018951F93CA
:101D7000CF93DF93CDB7DEB7AA970FB6F894DEBF47
:101D80000FBECDBFE0E7F2E088E08E0F9091F1004A
:101D900091938E13FBCF0E94380A8091E80083FF55
:101DA0001FC18091700290917102492F50E04A301A
:101DB000510508F015C1FA01E65CFF4F0C94A5250A
:101DC000803881F0823809F00BC1809174028F70E5
:101DD0008093E9008091EB0085FB882780F91092C1
:101DE000E90006C080916C0290916D0291118260B1
:101DF0009091E800977F9093E8008093F100109213
:101E0000F100C8C0282F2D7F09F0EAC0882319F0FF
:101E1000823061F0E5C080917202813009F0E0C04B
:101E2000933009F080E080936D022BC080917202A4
:101E3000811127C0809174028F7009F4D1C0809302
:101E4000E9002091EB0020FF1CC0933021F4809129
:101E5000EB00806214C09091EB0090619093EB00D6
:101E600021E030E0A90102C0440F551F8A95E2F736
:101E70004093EA001092EA008091EB008860809322
:101E8000EB001092E9008091E800877F86C0811105
:101E9000A7C0109172021F778091E3008078812B98
:101EA0008093E3008091E800877F8093E8000E94A0
:101EB000100D8091E80080FFFCCF8091E3008068E6
:101EC0008093E300111102C082E001C083E080939F
:101ED0006F0286C08058823008F082C08091720202
:101EE000909173028C3D53E0950779F583E08A83E6
:101EF0008AE289834FB7F894DE01139620E03EE032
:101F000051E2E32FF0E050935700E49120FF03C02B
:101F1000E295EF703F5FEF708E2F90E0EA3010F0A7
:101F2000C79601C0C0968D939D932F5F243149F7CA
:101F30004FBF8091E800877F8093E8006AE270E0FD
:101F4000CE0101960E941D0C14C0AE014F5F5F4F81
:101F5000609174020E94640BBC01892B09F440C09B
:101F60009091E800977F9093E80089819A810E9480
:101F70007D0C8091E8008B778093E80031C0803839
:101F800079F58091E800877F8093E80080916B026B
:101F90008093F1008091E8008E778093E8000E94A2
:101FA000100D1EC081111CC0909172029230C0F4BD
:101FB0008091E800877F8093E80090936B020E94F5
:101FC000100D80916B02811106C08091E30087FDA6
:101FD00002C081E001C084E080936F020E94240A65
:101FE0008091E80083FF0AC08091E800877F80939A
:101FF000E8008091EB0080628093EB00AA960FB618
:10200000F894DEBF0FBECDBFDF91CF911F91089531
:1020100090937D0180937C010895E0917C01F09183
:102020007D01309721F00190F081E02D099480E04E
:102030000895EF92FF920F931F93CF93DF93E09158
:102040007C01F0917D013097B1F18C010280F38128
:10205000E02D099580915A0282FF2DC080FF04C0B7
:1020600082EB93E00E945505E80118E08CEAE82E27
:1020700083E0F82E80915A0280FF0BC088811F9266
:102080008F93FF92EF920E94EE050F900F900F90AA
:102090000F90115021961111EDCF80915A0280FFBF
:1020A0000AC08AEA93E0DF91CF911F910F91FF90D0
:1020B000EF900C945505DF91CF911F910F91FF90F8
:1020C000EF900895E0917C01F0917D01309721F02F
:1020D0000480F581E02D09940895CF93DF93EC01FE
:1020E00080917A0190917B01C817D90709F1D093AB
:1020F0007B01C0937A01E0917C01F0917D013097E2
:10210000B9F00680F781E02DCE01099580915A0241
:1021100082FF0EC080FF0CC0DF93CF938CE993E069
:102120009F938F930E94EE050F900F900F900F904A
:10213000DF91CF910895CF93DF93EC0180917801E7
:1021400090917901C817D90709F1D0937901C0930B
:102150007801E0917C01F0917D013097B9F0008425
:10216000F185E02DCE01099580915A0282FF0EC0C3
:1021700080FF0CC0DF93CF938CE893E09F938F9305
:102180000E94EE050F900F900F900F90DF91CF916E
:1021900008950C94F7050E94E01C0C940706BF926A
:1021A000CF92DF92EF92FF920F931F93CF93DF9323
:1021B00000D000D01F92CDB7DEB70E9480060FE797
:1021C00011E0F12C8F2D0E94F905B82EF801C08086
:1021D000C82639F4F3940F5F1F4FF0E1FF12F2CFDE
:1021E00030C080915A0281FD0E947411D12CEE24DE
:1021F000E3948E2D8C21F9F0D982FA8281E09E2D14
:102200009B2109F480E08B830E94E91C8160782F78
:102210009D838C8349815A816B818D810E94AA1193
:1022200049815A816B817C818D810E94631CF801F8
:1022300090819E259083D394EE0CF8E0DF12D9CFE5
:10224000C9CF8FEF89838A831B820E94E91C81603A
:10225000782F9D838C8349815A816B818D810E9467
:10226000AA110E94621C0E94B61F10917E010E945A
:102270000D10181741F10E940D1080937E0190916E
:102280005A0292FF0EC090FF0CC01F928F938DEBED
:1022900093E09F938F930E94EE050F900F900F9005
:1022A0000F9080917E010F900F900F900F900F90E4
:1022B000DF91CF911F910F91FF90EF90DF90CF9022
:1022C000BF900C94741C0F900F900F900F900F9074
:1022D000DF91CF911F910F91FF90EF90DF90CF9002
:1022E000BF9008950C94E206EF92FF920F931F9314
:1022F000CF93DF9386ED93E00E945505C0E0D0E0D8
:1023000087E2E82E81E0F82E08EC13E08C2F0E9483
:10231000F9050E94501CFF92EF921F928F93DF935A
:10232000CF931F930F930E94EE0521968DB79EB712
:1023300008960FB6F8949EBF0FBE8DBFC031D10571
:1023400029F7DF91CF911F910F91FF90EF900895A2
:1023500008950895CF93DF93CDB7DEB72B970FB6CF
:10236000F894DEBF0FBECDBF942F4F83252F588723
:1023700069877A878B874A855B85452B21F02F3FBC
:1023800009F59F3FF9F4DE01119686E0FD011192F7
:102390008A95E9F785E0FE01379601900D928A95BE
:1023A000E1F749815A816B817C818D819E810E94F8
:1023B000C9182B960FB6F894DEBF0FBECDBFDF91C4
:1023C000CF9108954F81588569857A858B850E94C4
:1023D000631CD9CFCF93882309F465C0C82F8CEF35
:1023E0008C0F813A20F080E58C0F8E3248F48C2FD0
:1023F0000E94E222811157C08C2F0E94AC1B0CC09E
:1024000080E28C0F883058F4C77081E001C0880FDB
:10241000CA95EAF70E94EB1BCF910C94251C8BE523
:102420008C0F833078F4C53A29F0C63A31F083E84E
:1024300090E005C081E890E002C082E890E0CF9192
:102440000C946D1088E58C0F853168F5C83A89F0D9
:10245000C93A91F0CA3A99F0CB3AA1F0CC3AA9F036
:10246000CD3AB1F0CE3AB9F0CF3AC1F080E090E089
:1024700017C082EE90E014C089EE90E011C08AEEA1
:1024800090E00EC085EB90E00BC086EB90E008C0BA
:1024900083EB90E005C084EB90E002C087EB90E016
:1024A000CF910C949B10CF910895882349F19CEF14
:1024B000980F913A20F090E5980F9E3218F40E9400
:1024C000C91B0DC090E2980F983058F4877091E0C6
:1024D00001C0990F8A95EAF7892F0E94F11B0C948D
:1024E000251C9BE5980F933020F480E090E00C943D
:1024F0006D10885A853120F480E090E00C949B1098
:102500000895882321F00E94EB1B0C94251C08954C
:10251000882321F00E94F11B0C94251C0895BF9282
:10252000CF92DF92EF92FF920F931F93CF93DF939F
:1025300000D000D000D0CDB7DEB725E0FC01DE0131
:10254000119601900D922A95E1F7FC01408151818D
:10255000028163817481258122952F706115710537
:1025600009F403C35F3F19F44F3F09F4FEC26C0145
:10257000862F7D836C83602F782F8D812E830E9420
:10258000291B182FB92E0E94281B0E94181AEB2D08
:10259000E295EF70F0E0EC5BFF4F2E810C94A525E7
:1025A0008B2D807F9B2D9F70F92E882319F0F2943C
:1025B00090EFF922002349F0FF2009F483C28F2D08
:1025C0000E94FE1B0E94251C7DC2812F0E94551275
:1025D000FF2009F4CAC28F2D0E94041C26960FB654
:1025E000F894DEBF0FBECDBFDF91CF911F910F9149
:1025F000FF90EF90DF90CF90BF900C94251C8B2D17
:10260000807F9B2D9F70F92E803219F0F29480EF1D
:10261000F822112319F0113009F12AC00023B1F07A
:102620008F2D222351F1213041F526960FB6F894D3
:10263000DEBF0FBECDBFDF91CF911F910F91FF90F5
:10264000EF90DF90CF90BF900C940E1C222319F0D6
:10265000213009F48AC20E94111C2DC00023F1F020
:10266000263008F082C20E94E81B8F2129F023C087
:102670000023F9F0211116C08F2D26960FB6F8947D
:10268000DEBF0FBECDBFDF91CF911F910F91FF90A5
:10269000EF90DF90CF90BF900C948112253008F01E
:1026A00064C209C0F601858180FF0CC28F708583EA
:1026B000E3CF21111CC28F2D83C12B2D269526958A
:1026C000237030E02115310521F021303105D1F0A2
:1026D0004CC2002321F0812F9B2D937002C080E01B
:1026E00090E026960FB6F894DEBF0FBECDBFDF9107
:1026F000CF911F910F91FF90EF90DF90CF90BF90FF
:102700000C946D10002321F0812F9B2D937002C03B
:1027100080E090E026960FB6F894DEBF0FBECDBFE6
:10272000DF91CF911F910F91FF90EF90DF90CF90AD
:10273000BF900C949B10812F002319F00E943C1E27
:1027400002C00E94A41E26960FB6F894DEBF0FBEEC
:10275000CDBFDF91CF911F910F91FF90EF90DF9050
:10276000CF90BF900C94291F8B2D837009F07BC0F4
:102770000111FBC1812F829586958770880F880F84
:10278000912F9F70C92ED12CE12CF12C082E04C062
:10279000CC0CDD1CEE1CFF1C0A94D2F714FF12C0F7
:1027A0004FE050E060E070E004C0440F551F661F2A
:1027B000771F8A95D2F7CB01BA0160957095809505
:1027C000909503C060E070E0CB012B2D26952695F7
:1027D0002370422F50E042305105D9F0433051056B
:1027E00069F16C297D298E299F294130510551F1CC
:1027F00026960FB6F894DEBF0FBECDBFDF91CF9106
:102800001F910F91FF90EF90DF90CF90BF900C94AD
:102810003D1A6C297D298E299F2926960FB6F8949A
:10282000DEBF0FBECDBFDF91CF911F910F91FF9003
:10283000EF90DF90CF90BF900C94571A0E943D1AF2
:10284000C701B60126960FB6F894DEBF0FBECDBF06
:10285000DF91CF911F910F91FF90EF90DF90CF907C
:10286000BF900C94231A002319F08B2D817001C0A6
:102870008695882309F479C1812F82958695877082
:10288000880F880F912F9F70C92ED12CE12CF12C2D
:10289000082E04C0CC0CDD1CEE1CFF1C0A94D2F7E1
:1028A00014FF12C04FE050E060E070E004C0440F3D
:1028B000551F661F771F8A95D2F7CB01BA01609525
:1028C00070958095909503C060E070E0CB012B2D52
:1028D000269526952370422F50E042305105D9F0BD
:1028E0004330510569F16C297D298E299F2941309A
:1028F000510551F126960FB6F894DEBF0FBECDBF3D
:10290000DF91CF911F910F91FF90EF90DF90CF90CB
:10291000BF900C94041B6C297D298E299F29269633
:102920000FB6F894DEBF0FBECDBFDF91CF911F91E0
:102930000F91FF90EF90DF90CF90BF900C94161BFB
:102940000E94041BC701B60126960FB6F894DEBF9D
:102950000FBECDBFDF91CF911F910F91FF90EF90F0
:10296000DF90CF90BF900C94F21A103FD1F128F471
:1029700080E4810F803250F0A0C0123F09F462C0A1
:1029800008F44BC0133F09F472C097C0F12FF071E7
:10299000FF2E8B2D8F71002351F00E948B1A812FF7
:1029A000FF2019F08295807F68CE8F7066CE0E94DE
:1029B000AC1A812FFF2019F08295807F01C08F70A3
:1029C00026960FB6F894DEBF0FBECDBFDF91CF9134
:1029D0001F910F91FF90EF90DF90CF90BF900C94DC
:1029E00088120023B1F0253008F0BFC08B2D8F7105
:1029F00026960FB6F894DEBF0FBECDBFDF91CF9104
:102A00001F910F91FF90EF90DF90CF90BF900C94AB
:102A1000D11A263008F0A9C0E9CF0023A9F08B2DE8
:102A20008F7126960FB6F894DEBF0FBECDBFDF9133
:102A3000CF911F910F91FF90EF90DF90CF90BF90BB
:102A40000C948B1A002359F38B2D8F7126960FB699
:102A5000F894DEBF0FBECDBFDF91CF911F910F91D4
:102A6000FF90EF90DF90CF90BF900C94AC1A0023B2
:102A700099F08B2D8F7126960FB6F894DEBF0FBE9E
:102A8000CDBFDF91CF911F910F91FF90EF90DF901D
:102A9000CF90BF900C94761A26960FB6F894DEBFAE
:102AA0000FBECDBFDF91CF911F910F91FF90EF909F
:102AB000DF90CF90BF900C94711A0023A9F02223CD
:102AC00009F4ADCF812F26960FB6F894DEBF0FBE66
:102AD000CDBFDF91CF911F910F91FF90EF90DF90CD
:102AE000CF90BF900C94EA11222309F4ADCF812F2F
:102AF00026960FB6F894DEBF0FBECDBFDF91CF9103
:102B00001F910F91FF90EF90DF90CF90BF900C94AA
:102B100055124B2D4F70612FC6010E94B21D269693
:102B20000FB6F894DEBF0FBECDBFDF91CF911F91DE
:102B30000F91FF90EF90DF90CF90BF900C947119A0
:102B40004B2D4F70612FC60126960FB6F894DEBF4D
:102B50000FBECDBFDF91CF911F910F91FF90EF90EE
:102B6000DF90CF90BF900C94B51D26960FB6F894C9
:102B7000DEBF0FBECDBFDF91CF911F910F91FF90B0
:102B8000EF90DF90CF90BF9008950E940B1C0E94A1
:102B9000DA1B0E94251C0E945D200E94291F80E0F4
:102BA00090E00E946D1080E090E00C949B100E94D9
:102BB000FB1B0C94C515CF93DF9300D000D01F9260
:102BC000CDB7DEB7942F4983252F5A836B837C833F
:102BD0008D834C815D81452B39F12F3F11F49F3F4F
:102BE00019F149815A816B817C818D810E94291B59
:102BF000292F22952F7030E02C30310504F52A3032
:102C000031055CF4225031092230310568F4853AEF
:102C100080F4843090F4823080F0883E38F4803E36
:102C200060F48450813A48F080E014C0803FE1F7BE
:102C300004C090E2980F983080F781E00BC02C30F0
:102C4000310521F493FB882780F904C02F3031052A
:102C5000C9F3EACF0F900F900F900F900F90DF9174
:102C6000CF910895CF93DF9300D000D01F92CDB7BE
:102C7000DEB70F900F900F900F900F90DF91CF91D4
:102C80000895CF93DF9300D000D000D0CDB7DEB74A
:102C900026960FB6F894DEBF0FBECDBFDF91CF9161
:102CA0000895CF93DF93C0918F0180919001C81751
:102CB000A1F0D0E0CE0166E070E00E947425FC0136
:102CC000EF56FE4F408151816281738184819581ED
:102CD0000E9441162196C770E8CFDF91CF910895E9
:102CE0004091C1015091C2016091C3017091C40132
:102CF0008091C5019091C6010C944116CF93DF934A
:102D00008091C60182958F7009F05CC08091C301EB
:102D1000882309F457C020918F01D09190014091F0
:102D2000C101C091C201E091C401F091C5012D170C
:102D300009F448C030E0309709F440C0CF3F11F4A7
:102D40004F3FE1F1C90166E070E00E947425DC01AB
:102D5000AF56BE4F11968C911197C8132FC08C910E
:102D600048132CC012968C911297811127C013968C
:102D70008D919C9114978E179F0708F401978E1BD5
:102D80009F0B883C9105D0F48091C6018F708061C3
:102D90008093C601C90166E070E00E947425FC01C1
:102DA000EA56FE4F90819F709061908381EC91E094
:102DB0000E948F12DF91CF910C9451162F5F3F4FDD
:102DC0002770B5CFDF91CF910895BF92CF92DF9258
:102DD000EF92FF920F931F93CF93DF93CDB7DEB7A0
:102DE00061970FB6F894DEBF0FBECDBF7C0185E0C2
:102DF000F701DE011D9601900D928A95E1F7D7014A
:102E00004C9111962C9111971296DC901297139673
:102E10000D911C9114975091C1016091C201809154
:102E2000C4019091C501009709F481C16F3F19F465
:102E30005F3F09F47CC1B090C301BB2009F4CCC052
:102E40003091C6010817190728F0F801E81BF90BA3
:102E5000CF0104C080959095800F911FCC24C3941E
:102E6000883C910588F0C12C307F09F0D4C0702FC8
:102E7000198B088B522F6D2D89890E94321681EC97
:102E800091E00E948F12BDC0832F807F09F04AC05D
:102E9000621314C0541312C0D11010C03F703061BF
:102EA0003093C6010E94701681EC91E00E948F124F
:102EB0008091C601D70115968C9332C0011511057A
:102EC00031F12F3F11F44F3F11F1CD2CD1101FC024
:102ED000E0918F0130919001E31709F462C0F0E0B6
:102EE000CF0166E070E00E947425DC01AF56BE4F52
:102EF00011968C911197281307C08C91481304C028
:102F000012968C91811103C03196E770E5CFCD2CDC
:102F1000DD2009F42DC18091C60181608093C60136
:102F2000C12C26C1621308C0541306C0D11004C0BE
:102F30008091C601D701CEC04D872E87DF86702FC6
:102F4000198B088B522F6D2D89890E94DB158823E0
:102F500009F43EC0DD20E1F12091C601822F829567
:102F60008F7090E0029774F08091C1019091C2013E
:102F700098878F8319861B870A872C87CE0107962F
:102F80000E948F1286E0F701A1ECB1E001900D9252
:102F90008A95E1F70E947E160E947016CC24C39495
:102FA000E7C0702F198B088B522F60E089890E942F
:102FB000291B292F22952F7030E0223031050CF08B
:102FC000CBC09F7009F0C5C0805E883008F4D0C0C7
:102FD000C7010E948F12E2CF0817190708F458C0E2
:102FE000F801E81BF90BCF01883C910508F455C0A6
:102FF000C12C702F198B088B522F6D2D89890E943F
:103000003216E1ECF1E086E0DF011D928A95E9F7E6
:103010000E947016ADC0621314C0541312C0D110B8
:1030200010C08091C601F7018583C7010E948F12ED
:1030300086E0E1ECF1E0DF011D928A95E9F7CB2C07
:1030400097C04D872E87DF86702F198B088B522FE4
:103050006D2D89890E94DB15882309F4B9CFDD2005
:1030600009F4B6CF2091C601822F82958F7090E02F
:1030700002970CF487CF8091C1019091C2019A838D
:1030800089831B821D830C832E83CE01019678CF0A
:1030900080959095800F911FA7CFCD2CDD2009F44E
:1030A00097CF62132EC054132CC02091C60120FD6F
:1030B0001FC0822F82958F70D9F0D70115962C935F
:1030C00015978F3049F08F5F982F9295907F822FC0
:1030D0008F70892B15968C93C7010E948F1286E002
:1030E000F701A1ECB1E001900D928A95E1F790CF44
:1030F00086E0F701A1ECB1E001900D928A95E1F72D
:1031000037C04D872E87DF86702F198B088B522F83
:103110006D2D89890E94DB15811134CF8091C60104
:1031200081608093C601C7010E948F1221C0DD20FB
:1031300009F44ECF4D872E87DF86702F198B088BB1
:10314000522F6D2D89890E94DB15882309F440CF09
:1031500019CF811139CF0CC0243031050CF038CF94
:103160009F7009F431CFF7019581907F09F02CCF42
:103170008C2D61960FB6F894DEBF0FBECDBFDF91E8
:10318000CF911F910F91FF90EF90DF90CF90BF9064
:103190000895CF93DF93CDB7DEB72C970FB6F89491
:1031A000DEBF0FBECDBF4F83588769877A878B8775
:1031B0009C87CE0107960E94E516882371F08F81C7
:1031C00098852A853B85232B09F43FC09F3F09F052
:1031D00068C08F3F09F065C038C086E0FE013796B1
:1031E000DE01119601900D928A95E1F76F81788545
:1031F000EA85FB85309749F17F3F11F46F3F29F154
:103200008091900190E09C012F5F3F4F2770332702
:1032100040918F0150E02417350709F44BC06983B2
:103220007A83FD83EC8366E070E00E947425DC0104
:10323000AF56BE4F96E0FE01319601900D929A95E1
:10324000E1F7209390010E94511680918F01909197
:1032500090018917E9F190E066E070E00E94742522
:103260008F569E4F0E94E516882391F180918F0121
:1032700090E066E070E00E947425FC01EF56FE4F7E
:103280004081518162817381848195810E944116C0
:1032900080918F0190E001968770992780938F012C
:1032A000D4CF4F81588569857A858B859C850E940E
:1032B0004116CBCF0E94D7151092900110928F012A
:1032C000E1ECF1E086E0DF011D928A95E9F7BDCFE0
:1032D0002C960FB6F894DEBF0FBECDBFDF91CF9115
:1032E0000895DF92EF92FF920F931F93CF93DF9396
:1032F000FC01892B09F48AC0E12CF12CDD24D39444
:10330000EF0121968491853709F461C058F4843720
:1033100008F04EC0843008F06AC08130D1F08230AD
:1033200071F174C0883709F45DC050F4863709F430
:1033300055C0873709F06AC08E2D0E94F81B54C013
:103340009CE7980F903708F061C08F770E94551264
:1033500050C08F010E5F1F4FFE01849190E2980FC5
:10336000983050F48770FD2D01C0FF0F8A95EAF761
:103370008F2F0E94FE1B14C00E94EA1113C08F0100
:103380000E5F1F4FFE01C49180E28C0F883060F405
:10339000C7708D2D01C0880FCA95EAF70E94041CE2
:1033A0000E94251CE80125C08C2F0E945512FACFDF
:1033B0009F012E5F3F4FFE01C491CC2369F08FE93E
:1033C0009FE00197F1F700C00000C150F6CF9F01C8
:1033D0002E5F3F4FFE01F490E9010BC00E94E81BF5
:1033E000E82E07C00E94FB1B0E94251C02C00E9401
:1033F000EA118F2D882341F0EFE9FFE03197F1F7D3
:1034000000C000008150F6CFFE017ACFDF91CF914E
:103410001F910F91FF90EF90DF9008956093470206
:10342000709348028093490290934A020C94731C53
:10343000089560934B0270934C0280934D029093D9
:103440004E020C94721C0F931F9300914B0210912B
:103450004C0220914D0230914E02602B712B822B39
:10346000932B60934B0270934C0280934D02909388
:103470004E021F910F910C94721C0F931F93009199
:103480004B0210914C0220914D0230914E0260236C
:1034900071238223932360934B0270934C02809399
:1034A0004D0290934E021F910F910C94721C0F933A
:1034B0001F9300914B0210914C0220914D023091CC
:1034C0004E02602771278227932760934B027093E7
:1034D0004C0280934D0290934E021F910F910C94D9
:1034E000721C60E070E0CB010C940E1A0F931F93D6
:1034F00041E050E060E070E08A019B0104C0000FF1
:10350000111F221F331F8A95D2F7C901B8011F91DD
:103510000F910C940E1A0F931F9341E050E060E05E
:1035200070E004C0440F551F661F771F8A95D2F7BD
:103530008091470290914802A0914902B0914A02BD
:103540008A019B01082B192B2A2B3B2BC901B8019F
:103550001F910F910C940E1A0F931F9341E050E0AE
:1035600060E070E004C0440F551F661F771F8A9506
:10357000D2F7409550956095709580914702909153
:103580004802A0914902B0914A028A019B01082396
:1035900019232A233B23C901B8011F910F910C94D1
:1035A0000E1A0F931F9341E050E060E070E004C0FA
:1035B000440F551F661F771F8A95D2F780914702E7
:1035C00090914802A0914902B0914A028A019B0160
:1035D000082719272A273B27C901B8011F910F91F6
:1035E0000C940E1A0F931F930091470210914802FA
:1035F0002091490230914A02602B712B822B932B30
:103600001F910F910C940E1A0F931F930091470274
:10361000109148022091490230914A02602371239F
:10362000822393231F910F910C940E1A0F931F93D3
:1036300000914702109148022091490230914A02BC
:1036400060277127822793271F910F910C940E1AE0
:1036500008958F929F92AF92BF92DF92EF92FF9266
:103660000F931F93CF93DF9300D000D01F92CDB75D
:10367000DEB76B837C838D838A018C819D81892B4E
:1036800021F01F3F29F44F3F19F480E090E053C030
:103690008B81882309F43CC080904B0290904C02AF
:1036A000A0904D02B0904E02809147029091480246
:1036B000A0914902B0914A02882A992AAA2ABB2AD3
:1036C0002FE1E22EF12CD501C4010E2C04C0B695D9
:1036D000A795979587950A94D2F780FF07C0DE2CAF
:1036E000B8018E2D0E94831D019729F481E0E81A0C
:1036F000F10848F7D12CE12FF0E093E0EE0FFF1F27
:103700009A95E1F7E00FF11DE953FE4FD0820CC00E
:10371000E12FF0E083E0EE0FFF1F8A95E1F7E00F65
:10372000F11DE953FE4FD08009831A8369817A81A4
:103730008D2D0E94831D0F900F900F900F900F9072
:10374000DF91CF911F910F91FF90EF90DF90BF908D
:10375000AF909F908F90089520910B0130910C01B4
:10376000F90132969FEF40E05191581789F09F3F41
:1037700019F4511101C0942F4F5F4630A9F79F3FB4
:1037800039F0F901E90FF11D97FDFA95828308954B
:10379000089520910B0130910C01F9013296285FB8
:1037A0003F4F9081981301C010823196E217F307C2
:1037B000C1F7089581E090E0E0910B01F0910C01D8
:1037C000E80FF91F1082019688309105A9F7089536
:1037D00080915902089590915902892B8093590242
:1037E00008958095909159028923809359020895F4
:1037F00080935902089510925902089590915802A9
:10380000892B8093580208958095909158028923BE
:1038100080935802089510925802089580934F02A1
:10382000089510924F02089580910B0190910C0120
:10383000FC0131969C01285F3F4F80E091919111EE
:103840008F5FE217F307D1F70895E0910B01F09134
:103850000C01809159028083E0910B01F0910C01E1
:10386000908180915802892B808380914F02882318
:1038700061F0E0910B01F0910C019081892B808324
:103880000E94141C811110924F0280910B019091A3
:103890000C010C9419109093330180933201089518
:1038A0008295982F9C7C292F26952695982F937387
:1038B000990F990F922B892F8A7A86959575990F72
:1038C000892B08950895CF93DF9300D000D01F92E5
:1038D000CDB7DEB70F900F900F900F900F90DF9144
:1038E000CF910895089508950C94721180916F02FC
:1038F000843021F110925B0220E488E190E00FB661
:10390000F894A895809360000FBE2093600083B761
:10391000817F846083BF83B7816083BF78948895FB
:1039200083B78E7F83BF0FB6F894A895809160000F
:10393000886180936000109260000FBE0895CF935D
:103940000E94A8110E9480060E94A911C0E08C2F3D
:103950000E94F905811104C0CF5FC031C1F701C0D9
:1039600081E0CF9108950E94FF050C94D7151F9216
:103970000F920FB60F9211248F939F93AF93BF9323
:1039800080915B02811113C080915C0290915D0275
:10399000A0915E02B0915F024196A11DB11D80937E
:1039A0005C0290935D02A0935E02B0935F02BF91B0
:1039B000AF919F918F910F900FBE0F901F90189510
:1039C00082E084BD93E095BD9AEF97BD80936E0031
:1039D00008952FB7F89480915C0290915D02A091B8
:1039E0005E02B0915F022FBF08952FB7F8946091E7
:1039F0005C0270915D0280915E0290915F022FBF28
:103A00000895CF92DF92EF92FF920F931F932FB7FB
:103A1000F89440915C0250915D0260915E02709159
:103A20005F022FBF6A017B01EE24FF248C0120E09E
:103A300030E0C016D106E206F30610F441505109F9
:103A40009A01281B390BC9011F910F91FF90EF902C
:103A5000DF90CF9008951F920F920FB60F9211240E
:103A60008F939F93AF93BF9380915C0290915D027F
:103A7000A0915E02B0915F020196A11DB11D8093DD
:103A80005C0290935D02A0935E02B0935F02BF91CF
:103A9000AF919F918F910F900FBE0F901F9018952F
:103AA0000E94610DF8942FEF87EA91E62150804043
:103AB0009040E1F700C0000087E090EBDC018093CC
:103AC000780290937902A0937A02B0937B029CE0F3
:103AD00088E10FB6F894A895809360000FBE90938C
:103AE0006000FFCFE92FF0E093E0EE0FFF1F9A9503
:103AF000E1F7E80FF11DE855FF4F9491892F8F7082
:103B000092959F700895CF93C82FCB010E94721D8C
:103B1000492F90E0242F30E054E0220F331F5A95B4
:103B2000E1F7282B392B2038310519F480E090E09B
:103B300017C0EC2FF0E023E0EE0FFF1F2A95E1F70E
:103B40004770E40FF11D34E0EE0FFF1F3A95E1F7E7
:103B5000E80FF91FEE0FFF1FE050F849859194918F
:103B6000CF91089580E090E00895089580916202D9
:103B700080FF0CC08091100190E065E070E00E9431
:103B8000742595958795959587952EC081FF0AC0D8
:103B90008091100190E065E070E00E947425959599
:103BA000879522C082FF08C08091100190E065E0F7
:103BB00070E00E94742518C0209163022223D1F086
:103BC00030910F01231780F78091100190E065E09C
:103BD00070E00E947425622F70E00E947425632FAC
:103BE00070E00E949125CB018038910530F4009758
:103BF00031F0089585E090E008958FE7089581E021
:103C000008958091620280FF08C060910E0170E00B
:103C1000759567957595679523C081FF06C060917E
:103C20000E0170E0759567951BC082FF04C060911E
:103C30000E0170E012C0609163026623D1F0209102
:103C40000D016217A0F780910E0170E090E00E94D4
:103C50007425622F70E00E9491256038710528F468
:103C60006115710521F0862F08958FE7089581E091
:103C7000089561E070E0F4CF803F21F40E94B61D0A
:103C8000819504C0813F29F40E94B61D809366028D
:103C90000895823F21F40E94B61D819504C0833FA0
:103CA00029F40E94B61D809365020895893F19F496
:103CB0000E94011E05C08A3F31F40E94011E8195B9
:103CC0008093670208958B3F21F40E94011E819525
:103CD00004C08C3F29F40E94011E8093680208955D
:103CE000843F21F480916402816017C0853F21F4F4
:103CF00080916402826011C0863F21F48091640249
:103D000084600BC0873F21F480916402886005C005
:103D1000883F31F480916402806180936402089549
:103D20008D3F21F48091620281600BC08E3F21F4AF
:103D300080916202826005C08F3F29F48091620207
:103D40008460809362020895803F39F48091660216
:103D500087FF6CC01092660269C0813F29F4809190
:103D600066021816BCF362C090916502823F29F486
:103D700097FF5CC01092650259C0833F19F4191671
:103D8000CCF354C0893F41F48091670218160CF0BF
:103D90004DC0109267024AC08A3F29F480916702A1
:103DA00087FF44C0F6CF8B3F39F48091680287FFCC
:103DB0003DC0109268023AC08C3F29F4809168029D
:103DC0001816BCF333C0843F21F4809164028E7FC7
:103DD00017C0853F21F4809164028D7F11C0863F1A
:103DE00021F4809164028B7F0BC0873F21F4809186
:103DF0006402877F05C0883F31F4809164028F7E22
:103E00008093640213C08D3F21F4809162028E7F03
:103E10000BC08E3F21F4809162028D7F05C08F3FE1
:103E200029F4809162028B7F809362028091650207
:103E300081110EC08091660281110AC080916702D3
:103E4000811106C080916802811102C01092630244
:103E5000089580915A0283FF7EC08BE094E00E9417
:103E60005505809164021F928F9386E094E09F93A2
:103E70008F930E94EE0584E094E00E9455058091A6
:103E80006502282F082E000C330B3F938F9381E09F
:103E900094E09F938F930E94EE058FEF93E00E9432
:103EA000550580916602282F082E000C330B3F9396
:103EB0008F938CEF93E09F938F930E94EE058AEF90
:103EC00093E00E94550580916702282F082E000C70
:103ED000330B3F938F9387EF93E09F938F930E94D1
:103EE000EE0585EF93E00E94550580916802282F2A
:103EF000082E000C330B3F938F9382EF93E09F9338
:103F00008F930E94EE058FEE93E00E9455058091FD
:103F100063021F928F938CEE93E09F938F930E9486
:103F2000EE058AEE93E00E945505809162021F9291
:103F30008F9387EE93E09F938F930E94EE0584EE1C
:103F400093E00E9455058DB79EB74C960FB6F89436
:103F50009EBF0FBE8DBF84E692E00E9462100E9459
:103F6000E91C909361028093600208951F93CF93A0
:103F7000DF9380916002909161020E94011DFC011B
:103F800020916302222329F090911101892F90E062
:103F900007C08091120190E06AE070E00E947425F1
:103FA000E817F90708F485C080916502C0916602A0
:103FB000D091670210916802811107C0C11175C0CC
:103FC000D11173C0111171C074C02F3F19F02F5F50
:103FD00020936302181624F40E94B61D8093650294
:103FE0008091650287FF05C00E94B61D8195809370
:103FF00065021C1624F40E94B61D8093660280910F
:10400000660287FF05C00E94B61D819580936602F7
:1040100060916502662331F1C0916602CC2311F1F3
:10402000062E000C770B880B990B0E94732423E358
:1040300033E343E35FE30E94D7240E943B24609371
:1040400065026C2FCC0F770B880B990B0E947324A1
:1040500023E333E343E35FE30E94D7240E943B243E
:10406000609366021D1624F40E94011E809367026D
:104070008091670287FF05C00E94011E8195809391
:104080006702111624F40E94011E80936802809139
:10409000680287FF05C00E94011E81958093680217
:1040A000DF91CF911F910C94291F2F3F09F08FCFE3
:1040B00097CFDF91CF911F910895E4E6F2E085E07C
:1040C000DF011D928A95E9F7109263021092620255
:1040D00008958EE296E00E9455051F9281E08F932D
:1040E0001F9285E08F9380EE95E09F938F930E94BF
:1040F000EE050F900F900F900F900F900F90089576
:104100008330E9F128F4813061F0823009F10895BB
:10411000853009F462C008F449C0863009F474C0DF
:10412000089580911201262F30E0280F311D2F3F76
:10413000310524F4680F6093120103C08FEF809360
:104140001201809112011F928F9389E195E072C054
:1041500080911101262F30E0280F311D2F3F3105AE
:1041600024F4680F6093110103C08FEF8093110155
:10417000809111011F928F9387E095E05BC0809141
:104180001001262F30E0280F311D2F3F310524F478
:10419000680F6093100103C08FEF8093100180912E
:1041A00010011F928F9384EF94E044C080910F011F
:1041B000262F30E0280F311D2F3F310524F4680FE2
:1041C00060930F0103C08FEF80930F0180910F0167
:1041D0001F928F938FED94E02DC080910E01262FBA
:1041E00030E0280F311D2F3F310524F4680F609314
:1041F0000E0103C08FEF80930E0180910E011F927C
:104200008F9386EC94E016C080910D01262F30E04C
:10421000280F311D2F3F310524F4680F60930D01E5
:1042200003C08FEF80930D0180910D011F928F933A
:104230008BEA94E09F938F930E94EE050F900F906E
:104240000F900F900895833081F128F4813059F058
:104250008230D1F00895853009F449C0B8F1863034
:1042600009F456C0089580911201681720F4861B46
:104270008093120102C010921201809112011F92CC
:104280008F938CE994E054C080911101681720F459
:10429000861B8093110102C01092110180911101BF
:1042A0001F928F938AE894E043C0809110016817B1
:1042B00020F4861B8093100102C01092100180919F
:1042C00010011F928F9387E794E032C080910F0115
:1042D000681720F4861B80930F0102C010920F0113
:1042E00080910F011F928F9382E694E021C080910C
:1042F0000E01681720F4861B80930E0102C01092F5
:104300000E0180910E011F928F9389E494E010C0FA
:1043100080910D01681720F4861B80930D0102C067
:1043200010920D0180910D011F928F938EE294E007
:104330009F938F930E94EE050F900F900F900F9018
:104340000895CF93C82F1F928F9383E397E09F9395
:104350008F930E94EE0581E090E0A0E0B0E0BC0108
:10436000CD0104C0660F771F881F991FCA95D2F729
:104370000E94191A0F900F900F900F90CF910C94EC
:10438000D715CF93873288F58E3108F00BC18E3068
:1043900009F487C0D8F4873009F460C08B3009F481
:1043A0004FC0863009F002C180915A02817F8E7F12
:1043B00080935A0288E397E00E9455058CEF99E0BC
:1043C0000E94550581E080936A0246C0863109F457
:1043D000B0C020F4803109F47AC0E8C0893109F412
:1043E00091C08B3109F449C0E1C0883349F150F4E0
:1043F000893209F4D5C0853309F4D2C0873209F077
:10440000D5C0CEC0833409F4CBC028F48A3308F475
:10441000CDC08953C8C0883409F0C8C00E94D715E0
:104420008BEE99E00E9455052FEF83ED90E321502C
:1044300080409040E1F700C000000E94501D0CC079
:104440008FE597E041C082ED99E00E94550580918B
:104450005A02816080935A02C1E0ADC080915A0235
:10446000C82FC17080FFEFCF8EED99E00E945505F7
:1044700080915A02817F8E7F3FC090915A0291FBBA
:10448000CC27C0F981E0C827892FC0FB81F9809330
:104490005A02CC2319F085EC99E029C087EB99E00A
:1044A00013C090915A0292FBCC27C0F981E0C82733
:1044B000892FC0FB82F980935A02CC2319F088EA35
:1044C00099E015C088E999E00E945505C5CF909103
:1044D0005A0293FBCC27C0F981E0C827892FC0FB83
:1044E00083F980935A02CC2351F08CE899E00E9422
:1044F000550580915A02816080935A025CC08FE713
:1045000099E0E2CF80E799E00E94550588E499E0C0
:104510000E9455058EEF98E00E94550581ED98E0C8
:104520000E9455058CE898E00E9455058DE598E0BD
:10453000CBCF8FE498E00E9455050E940D101F928A
:104540008F9385E398E09F938F930E94EE0580916F
:104550000A011F928F938EE198E09F938F930E94A0
:10456000EE05809177011F928F938BE098E09F93E7
:104570008F930E94EE050E94F51C9F938F937F936B
:104580006F9384EF97E09F938F930E94EE058DB712
:104590009EB742960FB6F8949EBF0FBE8DBF5CCFFC
:1045A00080E001C08D510E94A12156CF82EF97E09B
:1045B0000E945505C0E08C2FCF91089580E00895AA
:1045C00080E00895CF93C82F80916A02813081F0F6
:1045D00020F0823009F44FC046C1E0910B01F09108
:1045E0000C018081813169F0823209F03EC109C03D
:1045F000E0910B01F0910C018081813111F0823248
:1046000061F48C2F0E94DE22811104C08C2F0E9445
:10461000C1212FC081E090E02CC08C2F0E94E022AD
:10462000811126C0C431E1F070F4CB3081F0C0318B
:10463000D1F40E9469208BE297E00E94550582E048
:1046400080936A0215C0C93259F0C83361F488E317
:1046500097E00E9455058FE297E00E94550508C03B
:1046600010926A0204C189E297E00E945505FFC0DA
:1046700081E08170FEC0C43228F5CE3108F0C1C09F
:10468000CB30A1F1D0F4C73009F0D3C08EE18093D4
:10469000120182E3809311018AE08093100184E18A
:1046A00080930F0188E080930E0188E280930D01D2
:1046B0008FEC95E00E945505BFC0C33149F1C4316C
:1046C000C1F0B7C0CB3409F4A9C028F4C93289F0CD
:1046D000C83361F0AEC0C13509F49EC0C23509F4DB
:1046E00099C0CE3409F0A5C06AE09EC00E9469203E
:1046F000A3C080916902882319F0109269029CC0BE
:104700008CED95E00E94550581E080936A02B1C06E
:1047100086EB95E00E94550584EA95E00E945505D8
:10472000809112011F928F9381EA95E09F938F935E
:104730000E94EE058FE995E00E9455058DE895E011
:104740000E945505809111011F928F938AE895E090
:104750009F938F930E94EE0588E895E00E9455058F
:1047600089E795E00E945505809110011F928F9373
:1047700086E795E09F938F930E94EE0584E795E08E
:104780000E94550583E695E00E94550580910F0132
:104790001F928F9380E695E09F938F930E94EE0582
:1047A0008EE595E00E94550589E495E00E94550547
:1047B00080910E011F928F9386E495E09F938F93D3
:1047C0000E94EE0584E495E00E9455058DE295E097
:1047D0000E94550580910D011F928F938AE295E00A
:1047E0009F938F930E94EE0588E295E00E94550505
:1047F0008DB79EB748960FB6F8949EBF0FBE8DBF7B
:104800001BC0CE51EC2FF0E0E85DFE4F808180931D
:10481000690212C061E003C061E006C06AE08091F5
:1048200069020E94802008C0809169020E942321B1
:1048300003C08DEC95E013C080916902882369F074
:104840001F928F9387EC95E09F938F930E94EE05C4
:104850000F900F900F900F9004C084EC95E00E9491
:10486000550581E006C010926A0280E002C080E037
:1048700000CFCF9108950E9442246894B1110C9406
:10488000D12408950E94B62488F09F5798F0B92F3C
:104890009927B751B0F0E1F0660F771F881F991F75
:1048A0001AF0BA95C9F714C0B13091F00E94D02423
:1048B000B1E008950C94D024672F782F8827B85F33
:1048C00039F0B93FCCF3869577956795B395D9F7CD
:1048D0003EF490958095709561957F4F8F4F9F4FD7
:1048E0000895E89409C097FB3EF4909580957095E3
:1048F00061957F4F8F4F9F4F9923A9F0F92F96E92C
:10490000BB279395F695879577956795B795F111A0
:10491000F8CFFAF4BB0F11F460FF1BC06F5F7F4F3D
:104920008F4F9F4F16C0882311F096E911C077234F
:1049300021F09EE8872F762F05C0662371F096E858
:10494000862F70E060E02AF09A95660F771F881F27
:10495000DAF7880F9695879597F9089557FD90583F
:10496000440F551F59F05F3F71F04795880F97FB33
:10497000991F61F09F3F79F08795089512161306ED
:104980001406551FF2CF4695F1DF08C0161617061C
:104990001806991FF1CF8695710561050894089551
:1049A000E894BB2766277727CB0197F908950E94E3
:1049B000E9240C9463250E94552538F00E945C255B
:1049C00020F0952311F00C944C250C9452250C9456
:1049D000D1240E94AE2478F39923C9F35523B9F367
:1049E000950F50E0551FAA27EE27FF27BB2700246D
:1049F0000894679520F4E20FF31FB41F0A1E220FDC
:104A0000331F441FAA1F6695A9F7779530F4F30F5B
:104A1000B41F0A1E121E08F46395330F441FAA1F09
:104A2000221F769599F7879520F4B40F0A1E121E5F
:104A3000631F440FAA1F221F331F8695A9F7862FD5
:104A4000712D602D11249F5750409AF0F1F088236A
:104A50004AF0EE0FFF1FBB1F661F771F881F915084
:104A60005040A9F79E3F510580F00C944C250C94C2
:104A7000D1245F3FE4F3983ED4F38695779567950C
:104A8000B795F795E7959F5FC1F7FE2B880F911DAE
:104A90009695879597F9089597F99F6780E870E054
:104AA00060E008959FEF80EC089500240A941616A4
:104AB000170618060906089500240A94121613060C
:104AC000140605060895092E0394000C11F488239A
:104AD00052F0BB0F40F4BF2B11F460FF04C06F5FB6
:104AE0007F4F8F4F9F4F08950024552704C0080E15
:104AF000591F880F991F009729F076956795B8F38D
:104B00007105B9F7802D952F0895991B79E004C0A0
:104B1000991F961708F0961B881F7A95C9F78095FC
:104B2000089597FB072E16F4009407D077FD09D05F
:104B30000E94AB2507FC05D03EF4909581959F4FD0
:104B40000895709561957F4F0895EE0FFF1F0590B2
:104B5000F491E02D0994AA1BBB1B51E107C0AA1FC9
:104B6000BB1FA617B70710F0A61BB70B881F991F0E
:104B70005A95A9F780959095BC01CD010895F894B8
:024B8000FFCF65
:104B8200C108B2098F095B092709015002280814DC
:104B92000A321E404D36224C03FF02C902A70233DD
:104BA200024C0265027E02000102030405060708A8
:024BB2000900F8
:106800008800EA44E944E244040005000600070069
:10681000080009000A000B000C000D000E000F001C
:1068200010001100120013001400150016001700CC
:10683000180019001A001B001C001D001E001F007C
:10684000200021002200230024002500260027002C
:10685000280029002A002B002C002D002E002F00DC
:10686000300031003200330034003500360037008C
:10687000380039003A003B003C003D003E003F003C
:1068800040004100420043004400450046004700EC
:10689000480049004A004B004C004D004E004F009C
:1068A000500051005200530054005500560057004C
:1068B000580059005A005B005C005D005E005F00FC
:1068C000600061006200630064006500850067008D
:1068D000680069006A006B006C006D006E006F005C
:1068E0007000710072007300890087008A008B00BD
:1068F000E000E100E200E300F1A1E500E600E700CE
:106900000100010001000100EA4401000100E2442D
:106910000100010001000100460001004A004B0097
:10692000010001004700480001000100E9440100A6
:106930000100010001000100010001003A003B00DC
:106940003C003D003E003F0040004100420043004B
:10695000010035004C0039000100440045005200A0
:1069600049000100010050004F0029004D004E0079
:1069700051000100680069006A006B006C006D0046
:106980006E006F0070007100720073000100010062
:1069900001000100010001000100010001004D00A3
:1069A0004A004E004B0001000100010001000100FF
:1069B00001000100010001000100010001000100CF
:1069C00001000100010001000100010001000100BF
:1069D00001000100010001000100010001000100AF
:1069E0000100010001000100490001000100010057
:1069F000010001000100010001000100010001008F
:00000001FF
